:0A170B0000010202030304040505B7
:10083C00E4F513F512F511F510C203C200C202C2A1
:10084C0001120A147E007F908E428F43754A007508
:10085C004BA27540007541AC7548007549DA754C72
:10086C0001754D0890E680E030E70E8540448541E7
:10087C0045854846854947800C85484485494585CA
:10088C004046854147EE54E070030209AD751400F3
:10089C007515807E007F908E168F17C3742E9FFF68
:1008AC0074019ECF2402CF3400FEE48F0F8E0EF520
:1008BC000DF50CF50BF50AF509F508AF0FAE0EADFD
:1008CC000DAC0CAB0BAA0AA909A808C3120DDE507B
:1008DC002AE515250BF582E514350AF58374CDF060
:1008EC00E4FAF9F8E50B2401F50BEA350AF50AE907
:1008FC003509F509E83508F50880C0E4F50BF50A6B
:10090C00F509F508AF0FAE0EAD0DAC0CAB0BAA0A8A
:10091C00A909A808C3120DDE5035AE0AAF0BE517B6
:10092C002FF582E5163EF583E0FDE5152FF582E502
:10093C00143EF583EDF0E4FAF9F8EF2401F50BEA37
:10094C003EF50AE93509F509E83508F50880B5855D
:10095C00144285154374902480FF740034FFFEC349
:10096C00E54B9FF54BE54A9EF54AC3E5459FF5459A
:10097C00E5449EF544C3E5479FF547E5469EF5469D
:10098C00C3E5419FF541E5409EF540C3E5499FF520
:10099C0049E5489EF548C3E54D9FF54DE54C9EF560
:1009AC004CD2E843D82090E668E04409F090E65C2D
:1009BC00E0443DF0D2AF90E680E020E105D2071292
:1009CC00148F90E680E054F7F0538EF8C203300198
:1009DC00051205A2C20130032912178B5024C20341
:1009EC001215E920001690E682E030E704E020E1E1
:1009FC00EF90E682E030E604E020E0E412151812F5
:070A0C00178D12175B80C774
:010A130022C0
:1005A20090E6B9E0700302067E1470030207272466
:1005B200FE70030207BC24FB70030206781470036A
:1005C20002067214700302066614700302066C249B
:1005D20005600302082812178F400302083490E6D0
:1005E200BBE024FE602C14604724FD6016146031C9
:1005F20024067066E54290E6B3F0E54390E6B4F077
:10060200020834E54A90E6B3F0E54B90E6B4F00216
:100612000834E54490E6B3F0E54590E6B4F002080C
:1006220034E54690E6B3F0E54790E6B4F0020834CC
:1006320090E6BAE0FF121544AA06A9077B01EA492F
:100642004B600DEE90E6B3F0EF90E6B4F0020834A2
:1006520090E6A0E04401F002083490E6A0E04401F4
:10066200F00208341216CD0208341217640208345C
:1006720012134E0208341216BB02083412179140AC
:100682000302083490E6B8E0247F602B14603C2417
:1006920002600302071DA200E433FF25E0FFA2026D
:1006A200E4334F90E740F0E4A3F090E68AF090E65E
:1006B2008B7402F0020834E490E740F0A3F090E675
:1006C2008AF090E68B7402F002083490E6BCE054A3
:1006D2007EFF7E00E0D3948040067C007D01800492
:1006E2007C007D00EC4EFEED4F240BF58274173E2C
:1006F200F583E493FF3395E0FEEF24A1FFEE34E6A9
:100702008F82F583E0540190E740F0E4A3F090E695
:100712008AF090E68B7402F002083490E6A0E0447E
:1007220001F0020834121793400302083490E6B82D
:10073200E024FE601D2402600302083490E6BAE061
:10074200B40105C20002083490E6A0E04401F002C0
:10075200083490E6BAE0705990E6BCE0547EFF7E21
:1007620000E0D3948040067C007D0180047C007D03
:1007720000EC4EFEED4F240BF58274173EF583E438
:1007820093FF3395E0FEEF24A1FFEE34E68F82F56E
:1007920083E054FEF090E6BCE05480FF1313135440
:1007A2001FFFE0540F2F90E683F0E04420F0020890
:1007B2003490E6A0E04401F08078121795507390CF
:1007C200E6B8E024FE60202402706790E6BAE0B446
:1007D2000104D200805C90E6BAE06402605490E6C4
:1007E200A0E04401F0804B90E6BCE0547EFF7E0026
:1007F200E0D3948040067C007D0180047C007D0073
:10080200EC4EFEED4F240BF58274173EF583E49314
:10081200FF3395E0FEEF24A1FFEE34E68F82F583ED
:10082200E04401F0800C120130500790E6A0E04451
:0908320001F090E6A0E04480F022
:01083B00229A
:0300330002008C3C
:04008C0053D8EF3224
:100090001201000200000040181601830000010256
:1000A00000010A06000200000040010009022E00C3
:1000B000010100A0FA0904000004FF000000070588
:1000C0000102400000070586020002000705020247
:1000D0000002000705810240000009022E00010114
:1000E00000A0FA0904000004FF0000000705010257
:1000F000400000070586024000000705020240009C
:100100000007058102400000040309040E035100AA
:1001100048005900430043004400140351004800C4
:1001200059002D003900530020002000200000005D
:03004300020E00AA
:03005300020E009A
:100E0000021648000216A50002168F0002166000A6
:100E1000021385000213BC00020DFF0002179700A9
:100E20000217980002179900020EB8000211BD00C7
:100E300002179A0002179B0002179C0002179D00E0
:100E400002179E000217970002179F000217A000CA
:100E50000217A1000217A2000217A3000217A400A4
:100E60000217A500021797000217970002179700B4
:100E70000217A6000217A7000217A8000217A90070
:100E80000217AA000217AB000217AC000217AD0050
:100E90000217AE000217AF000217B0000217B10030
:100EA0000217B2000217B3000217B4000217B50010
:080EB0000217B6000217B7009B
:1015180090E682E030E004E020E60B90E682E030DE
:10152800E119E030E71590E680E04401F07F147E91
:0C1538000012124290E680E054FEF02207
:1015E90090E682E044C0F090E681F0438701000074
:0415F90000000022CC
:10148F0030070990E680E0440AF0800790E680E09C
:10149F004408F07FDC7E0512124290E65D74FFF087
:0F14AF0090E65FF05391EF90E680E054F7F02263
:02154400A907F5
:10154600AE4CAF4D8F828E83A3E064037017AD015E
:1015560019ED7001228F828E83E07C002FFDEC3E18
:09156600FEAF0580DF7E007F006E
:01156F002259
:101242008E1E8F1F90E600E054187012E51F2401D5
:10125200FFE4351EC313F51EEF13F51F801590E64C
:1012620000E05418FFBF100BE51F25E0F51FE51E37
:1012720033F51EE51F151FAE1E7002151E4E6005CA
:061282001215FD80EE22B2
:1015FD007400F58690FDA57C05A3E582458370F901
:01160D0022BA
:10128800022A1A0002250000023A0000023D03F774
:10129800023600000222000002280000012E01018F
:1012A8003400013300013900013C00013200022CF6
:1012B8000000013FA0013100012700013500012F86
:0312C80000C1065C
:100A140090E6007412F090E6017443F00000009038
:100A2400E61074A0F000000000000090E611F00051
:100A3400000000000090E612F0000000E490E613CD
:100A4400F000000090E61474E0F0000000E490E68A
:100A540015F000000090E6047480F00000007402B9
:100A6400F00000007406F0000000E4F000000090C4
:100A7400E60274E6F000000090E60374F8F000006B
:100A84000090E670E04440F0000000E490E609F0D5
:100A940000000043B18043B20F43B24090E6180413
:100AA400F00000007411F000000090E61A7409F0E0
:100AB400000000E490E671F090E672F075B4FF7502
:100AC400B6FF75B67F43B18090E65EE04408F0005F
:100AD4000000E490E68DF090E65EE04404F000004F
:100AE40000E490E68FF053B2FED28112177443B142
:100AF40020E4FD7F801211367F647E001212427D55
:100B0400807F801211367F9A7E00121715C2047DF1
:100B14000D7F401211367D787F20121136E4FD7F5F
:100B240010121136E4FD7F081211367DC07F0212C7
:100B34001136E4FD7F0412113612176C90E67AE048
:100B440054FEF0E4FD7F9012159AE4F52F12160E70
:0A0B54001217001216EAE4F5302231
:09175B00300605120B5EC20622E5
:02178B00D32267
:02178D00D32265
:02178F00D32263
:10134E0090E680E030E71590E6247402F00000008D
:10135E00E490E625F0000000D2048013E490E62429
:10136E00F000000090E6257440F0000000C20490EA
:07137E00E6BAE0F538D322C6
:1016BB0090E740E538F0E490E68AF090E68B04F092
:0216CB00D32228
:0817640090E6BAE0F524D3225F
:1016CD0090E740E524F0E490E68AF090E68B04F094
:0216DD00D32216
:02179100D32261
:02179300D3225F
:02179500D3225D
:1001300090E6B9E0244B70030201BD147003020382
:100140009C24F570030203D714700302048424FD79
:1001500070030204CC14700302052F14700302050F
:10016000602414600302059EE490E68AF090E68B1A
:10017000F090E6A0E020E1F990E68BE0F5180000B1
:100180000090E6047480F000000053277FAD27FF45
:1001900012113690E6047406F0000000E4F090E7D7
:1001A00040E0FF7E00121242432780AD277F80127D
:1001B0001136D2061216F51216DF0205A0E490E6FB
:1001C0008AF090E68BF090E6A0E020E1F990E68BD3
:1001D000E0F518D3943F4024E4F51974402519F54F
:1001E00082E434E7F583E0FF74002519F582E434F6
:1001F00022F583EFF00519E519B440DF7F9A7E0000
:10020000121715902200E0FF7E0012171F902200A7
:10021000E0FF7E00121729902200E0FF7E001217F7
:1002200033902201E075F004A4FFAEF012173D9068
:100230002201E075F004A4FFAEF0121747902201EE
:10024000E075F004A4FFAEF0121751902205E0C350
:10025000940250035327CF902205E0B40208E5270B
:1002600054CF2410F527902205E0B40308E5275465
:10027000CF2420F527902205E0B40408E52754CFC9
:100280002430F527902221E070035327B7902221D4
:10029000E0B40108E527444054F7F527902221E017
:1002A000B40208E52754BF4408F527902226E070E1
:1002B000055327FD8003432702902207E0FD7F407E
:1002C000121136902208E0FD7F2012113690221183
:1002D000E0FD7F10121136902212E0FD7F0812110E
:1002E00036902223E0F534902220E0F5339022244A
:1002F000E0F53990222EE0F532902233E0F531A37B
:10030000E0F53C90223AE0F53F902206E0F52EE53C
:100310002E7003752E0190220BE0FEA3E07C0024DA
:1003200000F526EC3EF525A3E0FEA3E02400F53B16
:10033000EC3EF53A902207E0FEA3E02400F52BEC1A
:100340003EF52AA3E0FEA3E02400F53EEC3EF53D99
:10035000902211E0FEA3E02400F537EC3EF5369044
:10036000220FE0FEA3E02400F529EC3EF5289022C0
:100370002FE0FEA3E02400F523EC3EF52290221DA1
:10038000E0FD7F0212113690221EE0FD7F04121163
:1003900036902235E0540FF52F0205A0E4F51974CC
:1003A000002519F582E43422F583E0FF7440251915
:1003B000F582E434E7F583EFF00519E519B440DF81
:1003C000000000E490E68AF000000090E68B7440A4
:1003D000F01214EB0205A0E490E68AF090E68BF0B0
:1003E00090E6A0E020E1F990E68BE0F518D39400C8
:1003F00050030205A012177B120DFB7FE67E001250
:10040000124212177B7F047E00121242E4F519C3D8
:1004100074079519FF90E740E0FEA807088002C323
:1004200013D8FC20E005120DFB800312177B7F0A16
:100430007E001212427FE67E001216780519E51939
:10044000C3940840CAE4F519C374079519FF90E7EF
:1004500041E0FEA807088002C313D8FC20E0051283
:100460000DFB800312177B7F0A7E001212427FE68B
:100470007E001216780519E519C3940840CA1217B0
:100480007B0205A090E74074E7F0A37402F0A37428
:100490000DF0A37478F0A3740AF0A3740EF0E4A333
:1004A000F0A3F0A37483F0300405E4A3F080069079
:1004B000E74974FFF0000000E490E68AF0000000D5
:1004C00090E68B740AF01214EB0205A090E678E037
:1004D0004480F090E6797491F07F647E0012167883
:1004E00090E679E090E740F07F647E001216789005
:1004F000E679E090E741F07F647E0012167890E69E
:1005000079E090E742F07F647E0012167890E679F9
:10051000E090E743F090E678E04440F0000000E42B
:1005200090E68AF000000090E68B7404F08071E49D
:1005300090E68AF090E68BF090E6A0E020E1F9905A
:10054000E68BE0F518D39401405690E741E0FD7F3B
:100550004212159A90E740E0FD7F4E12159A8040B6
:10056000E490E68AF090E68BF090E6A0E020E1F9D6
:1005700090E68BE0F518D39400402590E740E070BA
:100580000312008090E740E0B40107E52F700312EA
:100590000DEF90E740E0B4020712160E8002D3225E
:0105A000C397
:0105A1002237
:10164800C0E0C083C082D2015391EF90E65D74017F
:08165800F0D082D083D0E03213
:10168F00C0E0C083C0825391EF90E65D7404F0D048
:06169F0082D083D0E0328E
:1016A500C0E0C083C0825391EF90E65D7402F0D034
:0616B50082D083D0E03278
:10138500C0E0C083C08290E680E030E70E8540442F
:10139500854145854846854947800C8548448549AA
:1013A500458540468541475391EF90E65D7410F0C1
:0713B500D082D083D0E032AA
:10166000C0E0C083C082D2035391EF90E65D74085E
:08167000F0D082D083D0E032FB
:1013BC00C0E0C083C08290E680E030E70E854044F8
:1013CC00854145854846854947800C854844854973
:1013DC00458540468541475391EF90E65D7420F07A
:0713EC00D082D083D0E03273
:010DFF0032C1
:01179700321F
:01179800321E
:01179900321D
:100EB800C0E0C0F0C083C082C0D075D000C000C000
:100EC80001C002C003C004C005C006C007C2AFE528
:100ED800306402605090E678E04480F090E67974DF
:100EE80091F07F647E0012167890E679E090E7C072
:100EF800F07F647E0012167890E679E090E7C1F002
:100F08007F647E0012167890E679E090E7C2F07F61
:100F1800647E0012167890E679E090E7C3F090E6D8
:100F280078E04440F090E7C0E530F000000090E63B
:100F38008F7404F00000005391EF90E65FE04404E2
:100F4800F0D2AFD007D006D005D004D003D002D05D
:0E0F580001D000D0D0D082D083D0F0D0E032D3
:1011BD00C0E0C0F0C083C082C0D075D000C000C0F8
:0D11CD0001C002C003C004C005C006C00779
:1011DA00C2AF90E6A1E020E1F990E780E0FF700459
:1011EA00F5218025BFFF07752100D205801BE4FD8C
:1011FA007F9012159A90E782E0FD7F4212159A902D
:10120A00E781E0FD7F4E12159A00000090E68DE41A
:0D121A00F05391EF90E65FE04408F0D2AF92
:10122700D007D006D005D004D003D002D001D0001B
:0B123700D0D0D082D083D0F0D0E032C5
:01179A00321C
:01179B00321B
:01179C00321A
:01179D003219
:01179E003218
:01179F003217
:0117A0003216
:0117A1003215
:0117A2003214
:0117A3003213
:0117A4003212
:0117A5003211
:0117A6003210
:0117A700320F
:0117A800320E
:0117A900320D
:0117AA00320C
:0117AB00320B
:0117AC00320A
:0117AD003209
:0117AE003208
:0117AF003207
:0117B0003206
:0117B1003205
:0117B2003204
:0117B3003203
:0117B4003202
:0117B5003201
:0117B6003200
:0117B70032FF
:10167800AD07AC06ED25E0FDEC33FCED4C6007ED65
:071688001D70011C80F5221A
:060F66008C1A8D1BA90787
:100F6C0075B6FF75B5FF53B07F53010753B1FE7FC4
:100F7C000A7E00121678E4FBFAC374029BFFE9A800
:100F8C0007088002C313D8FC30E00543B10280038C
:100F9C0053B1FD7F0A7E0012167843B10412167805
:100FAC0053B1FB1216780BBB00010AEB64034A70B9
:100FBC00C8E4FAFBC374099BFFE51BAE1AA807082B
:100FCC008005CEC313CE13D8F930E00543B10280AF
:100FDC000353B1FD7F0A7E0012167843B10412163A
:100FEC007853B1FB1216780BBB00010AEB640A4A6A
:100FFC0070C243B1017F0A7E0012167853B1FE1203
:02100C00167854
:01100E0022BF
:0A171500AD07AC06E4FF120F6622D8
:0A171F00AD07AC067F04120F66222E
:0A172900AD07AC067F05120F662223
:0A173300AD07AC067F06120F662218
:0A173D00AD07AC067F01120F662213
:0A174700AD07AC067F02120F662208
:0A175100AD07AC067F03120F6622FD
:041136008F1DA9055B
:10113A00C2A27F017E00121678E4FBFAAF03E9A887
:10114A0007088002C313D8FC30E004D2A18002C28F
:10115A00A17F017E00121678D2A0121678C2A012C0
:10116A0016780BBB00010AEB64084A70CFE4FAFB5D
:10117A00AF03E51DA807088002C313D8FC30E004BA
:10118A00D2A18002C2A17F017E00121678D2A012DB
:10119A001678C2A01216780BBB00010AEB64084A43
:1011AA0070CEC2A2D2A27F017E00121678C2A2120B
:0211BA001678A5
:0111BC002210
:03177F00C2A322E0
:03178200D2A322CD
:03178500C28322FA
:03178800D28322E7
:0717740012178212178822F0
:10162E0012177F7F0A7E0012167812178512178204
:0A163E00121678121788121678228F
:10157000E4F51CF51DE4FBFA12162E0BBB00010A64
:10158000BA02F5BBA8F2051DE51D7002051CC39447
:0915900004E51C6480948040DC39
:01159900222F
:0C0080007D107C277F017E0012130D22F2
:0C0DEF007D107C277F017E001212CC22B8
:10100F00E533B4010353B1DFE5317003120080E51E
:10101F0034706F752101902202E075F040A485F0C5
:10102F001CF51DAF217E00AC1CAD1D120DCCD3EFF6
:10103F009400EE940040117FEF7E03121242E51DE3
:10104F00151D7002151C80DB902203E0751C00F546
:10105F001DAF217E00AC1CAD1D120DCCD3EF940043
:10106F00EE940040117F007E01121242E51D151D06
:10107F007002151C80DB902204E0FF7E00121242EA
:10108F008009752101E521640160FAE531700312D1
:0A109F000DEFE533B4010343B12067
:0110A9002224
:100B5E007530011216F5C205E5317007E52F7003E9
:100B6E00120DEFE5294528700312157012100F3083
:100B7E000503020C74753002E4F518F519C3E51976
:100B8E009526E51895255029E4F51AF51BC3E51BA6
:100B9E00952E7480F8651A98500D12162E051BE5C9
:100BAE001B7002051A80E60519E5197002051880FA
:100BBE00CCE532D394004005AF321215C3E4F518DC
:100BCE00F519C3E519953EE518953D5030C28130B3
:100BDE0080FDD281E4F51AF51BC3E51B952E7480BA
:100BEE00F8651A98500D12162E051BE51B7002059E
:100BFE001A80E60519E5197002051880C5E4F51886
:100C0E00F519C3E5199526E51895255029E4F51A29
:100C1E00F51BC3E51B952E7480F8651A98500D12BE
:100C2E00162E051BE51B7002051A80E60519E5193F
:100C3E007002051880CCE536FD7F40121136E5377F
:100C4E00FD7F20121136C2813080FDD281E52AFD52
:100C5E007F40121136E52BFD7F20121136E4F53060
:060C6E0012160E12170021
:010C7400225D
:10159A00AB05AE0790E678E04480F090E679EEF08D
:1015AA007F647E00121678EBF012167890E678E0E7
:0915BA004440F07F64121678220F
:1012CC008C1E8D1FAB07AA06EB4A6034E5A0540FA9
:1012DC002460F5A0AF1FAE1E121678E5A0540F24A3
:1012EC00A0F5A0AF1FAE1E121678E5A0540F2480F7
:1012FC00F5A0AF1FAE1E121678EB1B70011A80C83A
:01130C0022BE
:10130D008C1E8D1FAB07AA06EB4A6034E5A0540F67
:10131D002480F5A0AF1FAE1E121678E5A0540F2441
:10132D0060F5A0AF1FAE1E121678E5A0540F245025
:10133D00F5A0AF1FAE1E121678EB1B70011A80C8F8
:01134D00227D
:10160E00E52FB40109E5A0540F2480F5A022E52FA3
:10161E00B40209E5A0540F2490F5A02253A00F2286
:0B16DF00E53554BFFD7F0112113622DB
:0B16EA00E5354440FD7F01121136225F
:0B16F500E53554DFFD7F0112113622A5
:0B170000E5354420FD7F011211362268
:040DFB0053B17F224F
:04177B0043B18022D4
:1014BE00E4F554F5551217007F327E0012124212D7
:1014CE0016F57F327E001212420555E55570020563
:0C14DE0054C39403E5546480948040D90A
:0114EA0022DF
:1014EB00E4F51AF51B1216EA7F327E001212421235
:1014FB0016DF7F327E00121242051BE51B700205C0
:0C150B001AC39403E51A6480948040D950
:0115170022B1
:1015C3008F1C432704AD277F80121136E51C600B67
:1015D300C2813080FDD281151C80F15327FBAD27DA
:0615E3007F801211362288
:08176C00E4F553D2E9D2AF22EB
:1013F30090E678E020E6F9C2E990E678E04480F0F0
:10140300EF25E090E679F090E678E030E0F990E6B9
:1014130078E04440F090E678E020E6F990E678E062
:0614230030E1D6D2E922FF
:10145D00A90790E678E020E6F9E553702390E67849
:10146D00E04480F0E925E090E679F08D4EAF03A9D8
:10147D0007754F018A508951E4F552755301D322F6
:02148D00C32278
:10142900A90790E678E020E6F9E553702590E6787B
:10143900E04480F0E925E0440190E679F08D4EAF73
:1014490003A907754F018A508951E4F55275530371
:04145900D322C322B5
:03004B00020C752F
:100C7500C0E0C083C082C085C084C086758600C0C0
:100C8500D075D000C000C001C002C003C006C007B7
:100C950090E678E030E206755306020D5F90E6783F
:100CA500E020E10CE55364026006755307020D5F11
:100CB500E55324FE605F14603624FE7003020D5078
:100CC50024FC7003020D5C24086003020D5FAB4F2A
:100CD500AA50A951AF5205528F82758300120D7D1E
:100CE50090E679F0E552654E7070755305806B900E
:100CF500E679E0AB4FAA50A951AE528E82758300BA
:100D0500120DAA755302E54E6401704E90E678E027
:100D15004420F08045E54E24FEB5520790E678E084
:100D25004420F0E54E14B5520A90E678E04440F0D0
:100D350075530090E679E0AB4FAA50A951AE528E9B
:100D450082758300120DAA0552800F90E678E04463
:100D550040F075530080037553005391DFD007D0E1
:100D650006D003D002D001D000D0D0D086D084D018
:080D750085D082D083D0E0326A
:030000000210AA41
:0C10AA00787FE4F6D8FD7581550210F146
:100D7D00BB010CE58229F582E5833AF583E022502B
:100D8D0006E92582F8E622BBFE06E92582F8E22275
:0D0D9D00E58229F582E5833AF583E493228F
:100DAA00F8BB010DE58229F582E5833AF583E8F07F
:100DBA00225006E92582C8F622BBFE05E92582C82B
:020DCA00F22213
:100DCC00EF8DF0A4A8F0CF8CF0A428CE8DF0A42E3B
:020DDC00FE22F5
:100DDE00EB9FF5F0EA9E42F0E99D42F0E89C45F06B
:010DEE0022E2
:1010B60002083CE493A3F8E493A34003F68001F20C
:1010C60008DFF48029E493A3F85407240CC8C3333B
:1010D600C4540F4420C8834004F456800146F6DF0A
:1010E600E4800B0102040810204080901288E47E00
:1010F600019360BCA3FF543F30E509541FFEE493FF
:10110600A360010ECF54C025E060A840B8E493A3C5
:10111600FAE493A3F8E493A3C8C582C8CAC583CAF0
:10112600F0A3C8C582C8CAC583CADFE9DEE780BEA8
:0112CB000022
:00000001FF
